:100000000C9490000C94B8000C94B8000C94B800B8
:100010000C94B8000C94B8000C94B8000C94B80080
:100020000C94B8000C94B8000C94B8000C94B80070
:100030000C94B8000C94B8000C94B8000C94B80060
:100040000C940A080C94B8000C94BD0A0C94EF0AA6
:100050000C94B8000C94B8000C94B8000C94B80040
:100060000C94B8000C94B8007F02810283028502D0
:10007000870289028B028D028F02F8050B061B0690
:100080002E06360662066A0672067A068106810622
:100090008106810681068106810681068106810628
:1000A0008106810681068106810681068106810618
:1000B00081068106810681068106F80504060B0685
:1000C0001B062E0636064906510659060000000892
:1000D000000201000003040700000000000000000F
:1000E00001020408102040800102040810200102CF
:1000F000040810200404040404040404020202029C
:10010000020203030303030300000000250028008C
:100110002B0000000000240027002A001D031F0BF5
:1001200011241FBECFEFD8E0DEBFCDBF11E0A0E0AD
:10013000B1E0E0ECFCE102C005900D92A635B107FC
:10014000D9F722E0A6E5B1E001C01D92A338B207BD
:10015000E1F711E0C0E2D1E004C02297FE010E9465
:10016000FE0DCC31D107C9F70E94630B0C945E0ED3
:100170000C94000061E0809114010E940F0961E07D
:10018000809112010E940F0961E0809110010E948C
:100190000F0961E080910E010E940F0961E08091DA
:1001A0000C010E940F0961E080910A010E940F0971
:1001B00061E0809108010E940F0961E080910601D1
:1001C0000E940F0961E0809104010E940F0961E023
:1001D000809102010E940F0926E040E855E260E0AC
:1001E00070E086EE91E00C94610A60E08091140169
:1001F0000E94480960E0809112010E94480960E075
:10020000809110010E94480960E080910E010E94D7
:10021000480960E080910C010E94480960E08091EB
:100220000A010E94480960E0809108010C94480985
:1002300060E0809114010E94480961E08091120100
:100240000E94480961E0809110010E94480960E025
:1002500080910E010E94480960E080910C010E948B
:10026000480960E080910A010E94480960E080919D
:1002700008010C94480961E0809114010E9448092A
:1002800061E0809112010E94480960E080911001B4
:100290000E94480961E080910E010E94480961E0D6
:1002A00080910C010E94480960E080910A010E943F
:1002B000480961E0809108010C94480961E080914F
:1002C00014010E94480961E0809112010E944809CE
:1002D00061E0809110010E94480961E080910E0167
:1002E0000E94480960E080910C010E94480960E08A
:1002F00080910A010E94480961E0809108010C94F4
:10030000480960E0809114010E94480961E08091F1
:1003100012010E94480961E0809110010E94480981
:1003200060E080910E010E94480960E080910C011C
:100330000E94480961E080910A010E94480961E039
:10034000809108010C94480961E0809114010E9499
:10035000480960E0809112010E94480961E08091A3
:1003600010010E94480961E080910E010E94480935
:1003700060E080910C010E94480961E080910A01CF
:100380000E94480961E0809108010C94480961E0ED
:10039000809114010E94480960E0809112010E943E
:1003A000480961E0809110010E94480961E0809154
:1003B0000E010E94480961E080910C010E944809E9
:1003C00061E080910A010E94480961E08091080182
:1003D0000C94480961E0809114010E94480961E091
:1003E000809112010E94480961E0809110010E94F1
:1003F000480960E080910E010E94480960E0809108
:100400000C010E94480960E080910A010E9448099D
:1004100060E0809108010C94480961E0809114012A
:100420000E94480961E0809112010E94480961E040
:10043000809110010E94480961E080910E010E94A4
:10044000480961E080910C010E94480961E08091B7
:100450000A010E94480961E0809108010C94480952
:1004600061E0809114010E94480961E080911201CD
:100470000E94480961E0809110010E94480961E0F2
:1004800080910E010E94480960E080910C010E9459
:10049000480961E080910A010E94480961E0809169
:1004A00008010C94480961E0809114010E944809F8
:1004B00061E0809112010E94480961E08091100181
:1004C0000E94480961E080910E010E94480961E0A4
:1004D00080910C010E94480961E080910A010E940C
:1004E000480960E0809108010C944809019789301F
:1004F0009105B8F48C5C9F4FFC010C94FC0D0C949E
:1005000018010C943B010C945E010C9481010C9435
:10051000A4010C94C7010C94EA010C940D020C94F4
:1005200030020C945302FC0164E670E00E94C60D98
:1005300070935B0160935A014CE946039001479F19
:10054000300D11242E0F3F1FC9016AE070E00E9498
:10055000C60D709359016093580146EF4603C001E0
:10056000479F900D1124820F931F90935701809302
:10057000560160E0809102010E9448098091560175
:1005800090915701823091051CF00E94760202C0C2
:100590000E9453026091000170910101882777FD4C
:1005A0008095982F0E94830861E0809102010E944B
:1005B000480960E0809104010E9448098091580137
:1005C00090915901009749F420915A0130915B01B3
:1005D000232B19F40E94F50002C00E94760260915C
:1005E000000170910101882777FD8095982F0E9466
:1005F000830861E0809104010E94480960E08091D5
:1006000006010E94480980915A0190915B01009770
:1006100019F40E94F50002C00E9476026091000168
:1006200070910101882777FD8095982F0E9483089B
:1006300061E0809106010C9448098AE691E00C94EF
:10064000830386EE91E00E947E09892B51F086EEAD
:1006500091E00E949709682F8AE691E00E948A063D
:10066000F0CF2EE531E042E651E066E671E08AE641
:1006700091E00E94600780915E0190915F01A091DE
:100680006001B0916101813D9740A105B10528F05D
:1006900010925D0110925C0126C08AE691E00E94F2
:1006A000E80720E030E0A9010E944F0D87FD0BC054
:1006B0008AE691E00E94E80720E030E040E05FE356
:1006C0000E949C0B0AC08AE691E00E94E80720E0A5
:1006D00030E040E05FE30E949B0B0E946C0C709343
:1006E0005D0160935C0180915C0190915D010197D7
:1006F00021F410925D0110925C0180915C01909157
:100700005D010C9493020F931F93FC010FEF1FEFF9
:100710009801008311832283338310861186128609
:1007200013864FEF59EC6AE97BE3408B518B628B68
:10073000738B408F518F628F738F40A351A362A33D
:1007400073A340A751A762A773A740AB51AB62AB9D
:1007500073AB00AF11AF22AF33AFDC01A05CBF4F72
:100760008FEF90E011969C938E9314960D931D93AA
:100770002D933C93139718960D931D932D933C93B3
:10078000139718961C9211961C92509682E08C93A7
:1007900011961C9211961C9211961C9211961D9204
:1007A0001D921D921C921397149611961C921E92E4
:1007B00012961D921C92EA5AFF4F10821F910F91C0
:1007C00008952FEB260F862F992787FD90952630C9
:1007D00010F4C79708956156663018F4875591094B
:1007E0000895C09708950F931F93FB0160E070E098
:1007F000CB01019120ED200F2A30A0F4AAE0B0E057
:100800009B01AC010E94020E112707FD1095212FBC
:10081000312F600F711F821F931F6053710981096F
:100820009109E7CF1F910F9108950F931F93CF93D5
:10083000FC01EA5AFF4FC1E020812D3219F0C0E0DF
:100840008F0103C08C01095A1F4FB8010E94F303A6
:100850009B01AC01A4E6B0E00E94020EF801DF01AA
:10086000219130ED320F3A30D0F32E3269F51196E6
:100870002C91119730ED320F3A3030F5332727FDA8
:100880003095205331094AE0429F8001439F100D6B
:100890001124222717FD2095322F600F711F821F10
:1008A000931F12960C9120ED200F2A3068F4112727
:1008B00007FD109500531109222717FD2095322FAF
:1008C000600F711F821F931FCC2339F09095809584
:1008D000709561957F4F8F4F9F4FCF911F910F91D3
:1008E00008954F925F926F927F928F929F92AF92F4
:1008F000BF92CF92DF92EF92FF92CF93DF93EC0102
:10090000CA5ADF4FBE010E94F3032B013C0124E6CB
:1009100030E040E050E00E94DA0D9B01AC0160EA5B
:1009200076E881E090E00E94B60D6B017C01FE014B
:10093000819190ED980F9A30D8F38E3219F5EF012E
:1009400080E1882E87E2982EA12CB12CA99180ED10
:100950008A0F8A30B8F4BB27A7FDB095D097A501C0
:1009600094010E940D0EC60ED71EE81EF91EC50189
:10097000B4012AE030E040E050E00E94DA0D490185
:100980005A01E4CFC701B6016D5F7F4F8F4F9F4F74
:1009900026E030E040E050E00E94DA0D69017A0183
:1009A000C301B20124E630E040E050E00E94DA0DDD
:1009B00060E472E48FE090E00E94B60DC60ED71E90
:1009C000E81EF91EC701B601DF91CF91FF90EF90AD
:1009D000DF90CF90BF90AF909F908F907F906F905F
:1009E0005F904F900895DB01FA018D91882319F0F3
:1009F00091918917D1F3992787FD90950895CF920A
:100A0000DF92EF92FF921F93CF93DF93EC01FC01F3
:100A1000EB5AFF4F1081112309F4A9C03196608170
:100A20000E94E103182FFE01E95AFF4F6081CE01B9
:100A30000E94E10340E1149F800D1124FE01EC5A55
:100A4000FF4F908189138AC074961081112309F495
:100A500058C1359680819181019691838083B597A5
:100A600080819181A281B381349780839183A28315
:100A7000B3833C9680819181A281B3813497808336
:100A80009183A283B383799680818823A1F18130F9
:100A900009F037C18C819D81AE81BF8188839983A4
:100AA000AA83BB838C859D85AE85BF858887998702
:100AB000AA87BB878C899D89AE89BF89888B998BD2
:100AC000AA8BBB8B8C8D9D8DAE8DBF8D888F998FA2
:100AD000AA8FBB8F8CA59DA5AEA5BFA588A799A7FA
:100AE000AAA7BBA78CA99DA9AEA9BFA988AB99ABA2
:100AF000AAABBBAB06C18CA19DA1AEA1BFA188A32F
:100B000099A3AAA3BBA38C819D81AE81BF81888359
:100B10009983AA83BB838C899D89AE89BF89888B81
:100B2000998BAA8BBB8B8C8D9D8DAE8DBF8D888F45
:100B3000998FAA8FBB8FFE01E05CFF4FDE01AE5B99
:100B4000BF4F8D919C91918380838CAD9DADAEAD57
:100B5000BFAD88AF99AFAAAFBBAFD3C0C159DF4F0C
:100B60008881998101969983888310E0CAC0FC012D
:100B7000EA59FF4F30818B599F4F7C0131111DC0C5
:100B80006E0196E5C90ED11C46E151E0B601CE01D9
:100B90000E94F304892B11F481E00CC04CE151E078
:100BA000B601CE010E94F304892B19F4F7011082DB
:100BB000A8C082E0D7018C93A4C0DC01EC91E230A4
:100BC00009F49FC0CE018A5A9F4FDC012C91222349
:100BD00009F497C0B0E2EB9FF0011124E32B3197A9
:100BE000E932F10508F08DC0E35CFF4F0C94FC0D79
:100BF000CE010E9415046C837D838E839F830E94A7
:100C00005408C85BDF4F12C0C859DF4F81E0213460
:100C100009F05DC05DC0CE010E9471046C8B7D8BBC
:100C20008E8B9F8B0E945408C05BDF4F6883798353
:100C30008A839B8366C0233509F063C08C899D89B4
:100C4000AE89BF89B095A095909581959F4FAF4F84
:100C5000BF4F8C8B9D8BAE8BBF8B53C0CE010E9440
:100C600071046C8F7D8F8E8F9F8F4BC0273509F05D
:100C700048C08C8D9D8DAE8DBF8DB095A095909503
:100C800081959F4FAF4FBF4F8C8F9D8FAE8FBF8F82
:100C900038C0CE010E9415046CA77DA78EA79FA720
:100CA00030C0CE010E9415046CAB7DAB8EAB9FAB08
:100CB00028C0BC01CE010E94F3036C877D878E871C
:100CC0009F871FC0C859DF4F81E021330CF480E0BB
:100CD000888317C00E94380ECE5BDF4F9927998317
:100CE00088830FC0CE010E9415046CAF7DAF8EAF1C
:100CF0009FAF07C0CE010E9415046CA37DA38EA3F5
:100D00009FA3812FDF91CF911F91FF90EF90DF90F4
:100D1000CF900895CF92DF92EF92FF920F931F939F
:100D2000CF93DF931F92CDB7DEB76C01262FFC0166
:100D3000E759FF4F40815181628173814F5F5F4F5F
:100D40006F4F7F4F40835183628373838C010959B6
:100D50001F4F8B5A9F4F7C01243281F12CF42A3093
:100D600069F02D30E9F50AC02A3241F02C32C1F584
:100D7000F601EC5AFF4F808182278083F801808141
:100D80008F3060F4F601E80FF11DEA5AFF4F108230
:100D9000C60129830E94FF04298101C080E0F60179
:100DA000EA59FF4F90819F5F9083F801108291E094
:100DB0002A3209F090E0F70190832AC0F8011082EE
:100DC000F601EA59FF4F108272971082719682E005
:100DD0008083F7011082F601E859FF4F108217C097
:100DE000F80180818E3048F491E0980F9083F601ED
:100DF000E80FF11DEA5AFF4F2083F701808181112E
:100E000006C0F601EC5AFF4F80818227808380E084
:100E10000F90DF91CF911F910F91FF90EF90DF9096
:100E2000CF900895CF92DF92EF92FF920F931F938E
:100E3000CF93DF93E9016115710551F0FC01C08882
:100E4000D188E288F388FB01C082D182E282F382FA
:100E50004115510551F0FC01C08CD18CE28CF38C12
:100E6000FA01C082D182E282F382209701F18C01E3
:100E7000045B1F4FF80180819181A281B3818F3F74
:100E80009F4FAF4FBF4F61F00E945408F80100819F
:100E9000118122813381601B710B820B930B03C084
:100EA0006FEF7FEFCB01688379838A839B83DF9128
:100EB000CF911F910F91FF90EF90DF90CF90089509
:100EC000AF92BF92CF92DF92EF92FF920F931F9358
:100ED000CF93DF93CDB7DEB728970FB6F894DEBF78
:100EE0000FBECDBF5B018A01AE014F5F5F4FBE01F8
:100EF0006B5F7F4F0E941207CD80DE80EF80F88409
:100F00008FEFC81689ECD8068AE9E8068BE3F80665
:100F100059F0C701B6010E949F0C20E034E244E77B
:100F200059E40E94040C04C060E070E08AE794E495
:100F3000F5016083718382839383FFEFCF16F9EC11
:100F4000DF06FAE9EF06FBE3FF0669F069817A81C3
:100F50008B819C810E949F0C20E034E244E759E49D
:100F60000E94040C04C060E070E08AE794E4F80199
:100F7000608371838283938328960FB6F894DEBFD3
:100F80000FBECDBFDF91CF911F910F91FF90EF90DA
:100F9000DF90CF90BF90AF900895FC0160A571A540
:100FA00082A593A56F3FF9EC7F07FAE98F07FBE372
:100FB0009F0749F00E949D0C20E030E048EC52E48D
:100FC0000E94040C089560E070E080E89FEB0895B3
:100FD000CF92DF92EF92FF920E94CD076B017C01CE
:100FE00020E030E040E85FEB0E94000C882349F0ED
:100FF00026E53EE04DEE5FE3C701B6010E94530DCA
:1010000004C060E070E080E89FEBFF90EF90DF901D
:10101000CF9008951F920F920FB60F9211242F9325
:101020003F938F939F93AF93BF938091DE019091F5
:10103000DF01A091E001B091E1013091DD0126E0F6
:10104000230F2D3720F40296A11DB11D05C029E8FC
:10105000230F0396A11DB11D2093DD018093DE01B6
:101060009093DF01A093E001B093E1018091E20150
:101070009091E301A091E401B091E5010196A11DD9
:10108000B11D8093E2019093E301A093E401B0933A
:10109000E501BF91AF919F918F913F912F910F905B
:1010A0000FBE0F901F9018952FB7F8946091DE0136
:1010B0007091DF018091E0019091E1012FBF0895CF
:1010C0003FB7F8948091E2019091E301A091E4018F
:1010D000B091E50126B5A89B05C02F3F19F00196F8
:1010E000A11DB11D3FBF6627782F892F9A2F620F50
:1010F000711D811D911D43E0660F771F881F991F89
:101100004A95D1F70895CF92DF92EF92FF92CF9355
:10111000DF936B017C010E946008EB01C114D104D4
:10112000E104F10489F00E949A0B0E9460086C1B94
:101130007D0B683E734090F381E0C81AD108E10846
:10114000F108C851DC4FEACFDF91CF91FF90EF90CB
:10115000DF90CF900895789484B5826084BD84B583
:10116000816084BD85B5826085BD85B5816085BDA2
:10117000EEE6F0E0808181608083E1E8F0E01082BB
:10118000808182608083808181608083E0E8F0E0FC
:10119000808181608083E1EBF0E0808184608083E6
:1011A000E0EBF0E0808181608083EAE7F0E080811D
:1011B0008460808380818260808380818E7F808351
:1011C0008081806880831092C1000895833081F00F
:1011D00028F4813099F08230A1F008958730A9F089
:1011E0008830B9F08430D1F4809180008F7D03C0C5
:1011F000809180008F7780938000089584B58F77E9
:1012000002C084B58F7D84BD08958091B0008F7732
:1012100003C08091B0008F7D8093B0000895CF937C
:10122000DF9390E0FC01E052FF4F2491FC01EC5071
:10123000FF4F8491882349F190E0880F991FFC01AA
:10124000EE5EFE4FA591B491885F9E4FFC01C59163
:10125000D4919FB7611108C0F8948C912095822396
:101260008C93888182230AC0623051F4F8948C9167
:10127000322F309583238C938881822B888304C0FE
:10128000F8948C91822B8C939FBFDF91CF9108951E
:101290000F931F93CF93DF931F92CDB7DEB7282F05
:1012A00030E0F901E453FF4F8491F901E052FF4F20
:1012B0001491F901EC50FF4F04910023C9F08823E9
:1012C00021F069830E94E6086981E02FF0E0EE0FCB
:1012D000FF1FE85FFE4FA591B4919FB7F8948C91E2
:1012E000611103C01095812301C0812B8C939FBF96
:1012F0000F90DF91CF911F910F910895FC01818D87
:10130000228D90E0805C9F4F821B91098F739927FB
:101310000895FC01918D828D981731F0828DE80F30
:10132000F11D858D90E008958FEF9FEF0895FC01EA
:10133000918D828D981761F0828DDF01A80FB11D0C
:101340005D968C91928D9F5F9F73928F90E0089530
:101350008FEF9FEF089585E19BE0892B49F080E0B6
:1013600090E0892B29F00E94150B81110C9400004C
:101370000895FC01848DDF01A80FB11DA35ABF4F52
:101380002C91848D90E001968F739927848FA68984
:10139000B7892C93A089B1898C9180648C93938DAB
:1013A000848D981306C00288F389E02D80818F7D9B
:1013B00080830895CF93DF93EC01888D8823C9F053
:1013C000EA89FB89808185FD05C0A889B9898C914E
:1013D00086FD0FC00FB607FCF5CF808185FFF2CFE9
:1013E000A889B9898C9185FFEDCFCE010E94B909FA
:1013F000E7CFDF91CF910895CF92DF92FF920F93C5
:101400001F93CF93DF931F92CDB7DEB76C0181E0BE
:10141000D60158968C9358975B969C915B975C96F7
:101420008C915C97981307C05096ED91FC91519761
:10143000808185FD2EC0F601038D10E00F5F1F4FE8
:101440000F731127F02EF601848DF81211C00FB61C
:1014500007FCF9CFD6015096ED91FC915197808110
:1014600085FFF1CFC60169830E94B9096981EBCF7D
:10147000838DE80FF11DE35AFF4F6083D6015B9621
:101480000C935B975296ED91FC915397808180620B
:101490000CC0D6015696ED91FC91579760835096FB
:1014A000ED91FC91519780818064808381E090E090
:1014B0000F90DF91CF911F910F91FF90DF90CF9010
:1014C0000895BF92CF92DF92EF92FF92CF93DF9376
:1014D000EC016A017B01B22E60E874E88EE190E0D5
:1014E000A70196010E94DA0D2150310941095109E5
:1014F0005695479537952795E889F98982E0808345
:10150000211580E1380798F0E889F989108260E4B4
:1015100072E48FE090E0A70196010E94DA0D21505D
:101520003109410951095695479537952795EC851D
:10153000FD853083EE85FF852083188EEC89FD893B
:10154000B082EA89FB89808180618083EA89FB8996
:10155000808188608083EA89FB89808180688083BC
:10156000EA89FB8980818F7D8083DF91CF91FF9015
:10157000EF90DF90CF90BF9008951F920F920FB61B
:101580000F9211242F938F939F93EF93FF93E091EA
:10159000F601F091F7018081E091FC01F091FD01ED
:1015A00082FD12C090818091FF018F5F8F73209127
:1015B0000002821751F0E091FF01F0E0EA51FE4F86
:1015C000958F8093FF0101C08081FF91EF919F91E2
:1015D0008F912F910F900FBE0F901F9018951F9213
:1015E0000F920FB60F9211242F933F934F935F9357
:1015F0006F937F938F939F93AF93BF93EF93FF93DB
:1016000086EE91E00E94B909FF91EF91BF91AF91F1
:101610009F918F917F916F915F914F913F912F910A
:101620000F900FBE0F901F90189586EE91E00E94CC
:101630007E0921E0892B09F420E0822F0895109281
:10164000E9011092E80188EE93E0A0E0B0E0809319
:10165000EA019093EB01A093EC01B093ED018AE4D1
:1016600091E09093E7018093E60185EC90E0909300
:10167000F3018093F20184EC90E09093F501809364
:10168000F40180EC90E09093F7018093F60181ECF7
:1016900090E09093F9018093F80182EC90E09093B0
:1016A000FB018093FA0186EC90E09093FD0180931A
:1016B000FC011092FF0110920002109201021092A0
:1016C0000202089508950E94AB080E94620B0E94D6
:1016D000BA00CBEAD9E00E9421032097E1F30E94EF
:1016E000AB09F9CFCF92DF92EF92FF920F931F9346
:1016F000CF93DF936C017A01EB01E60EF71E00E059
:1017000010E0CE15DF0561F06991D601ED91FC91F5
:101710000190F081E02DC6010995080F191FF1CF46
:10172000C801DF91CF911F910F91FF90EF90DF9053
:10173000CF90089508955058BB27AA270ED075C1A1
:1017400066D130F06BD120F031F49F3F11F41EF4DC
:101750005BC10EF4E095E7FB51C1E92F77D180F32F
:10176000BA17620773078407950718F071F49EF59E
:101770008FC10EF4E0950B2EBA2FA02D0B01B901ED
:1017800090010C01CA01A0011124FF27591B99F0F7
:10179000593F50F4503E68F11A16F040A22F232F03
:1017A000342F4427585FF3CF469537952795A79553
:1017B000F0405395C9F77EF41F16BA0B620B730BFA
:1017C000840BBAF09150A1F0FF0FBB1F661F771F6B
:1017D000881FC2F70EC0BA0F621F731F841F48F420
:1017E000879577956795B795F7959E3F08F0B3CFA6
:1017F0009395880F08F09927EE0F97958795089590
:10180000D9D008F481E008950CD00FC107D140F081
:10181000FED030F021F45F3F19F0F0C0511139C112
:10182000F3C014D198F39923C9F35523B1F3951B51
:10183000550BBB27AA2762177307840738F09F5FF1
:101840005F4F220F331F441FAA1FA9F333D00E2E60
:101850003AF0E0E830D091505040E695001CCAF7CD
:1018600029D0FE2F27D0660F771F881FBB1F261792
:1018700037074807AB07B0E809F0BB0B802DBF0165
:10188000FF2793585F4F2AF09E3F510568F0B6C07E
:1018900000C15F3FECF3983EDCF386957795679542
:1018A000B795F7959F5FC9F7880F911D9695879516
:1018B00097F90895E1E0660F771F881FBB1F621735
:1018C00073078407BA0720F0621B730B840BBA0BF3
:1018D000EE1F88F7E095089504D06894B111D9C03F
:1018E0000895BCD088F09F5790F0B92F9927B75131
:1018F000A0F0D1F0660F771F881F991F1AF0BA95D4
:10190000C9F712C0B13081F0C3D0B1E00895C0C0B2
:10191000672F782F8827B85F39F0B93FCCF38695C9
:1019200077956795B395D9F73EF490958095709526
:1019300061957F4F8F4F9F4F0895E89409C097FBA3
:101940003EF490958095709561957F4F8F4F9F4F96
:101950009923A9F0F92F96E9BB279395F6958795DA
:1019600077956795B795F111F8CFFAF4BB0F11F49D
:1019700060FF1BC06F5F7F4F8F4F9F4F16C0882344
:1019800011F096E911C0772321F09EE8872F762F7A
:1019900005C0662371F096E8862F70E060E02AF0BB
:1019A0009A95660F771F881FDAF7880F96958795A7
:1019B00097F90895990F0008550FAA0BE0E8FEEF7C
:1019C00016161706E807F907C0F012161306E40703
:1019D000F50798F0621B730B840B950B39F40A26FC
:1019E00061F0232B242B252B21F408950A2609F4DA
:1019F000A140A6958FEF811D811D089597F99F67DE
:101A000080E870E060E008959FEF80EC0895002486
:101A10000A941616170618060906089500240A9453
:101A200012161306140605060895092E0394000CD9
:101A300011F4882352F0BB0F40F4BF2B11F460FF68
:101A400004C06F5F7F4F8F4F9F4F089557FD905891
:101A5000440F551F59F05F3F71F04795880F97FB72
:101A6000991F61F09F3F79F087950895121613062C
:101A70001406551FF2CF4695F1DF08C0161617065B
:101A80001806991FF1CF8695710561050894089590
:101A9000E894BB2766277727CB0197F908958ADF5B
:101AA00008F48FEF08950BD0C0CFB1DF28F0B6DF78
:101AB00018F0952309F0A2CFA7CF1124EACFC6DFF3
:101AC000A0F3959FD1F3950F50E0551F629FF00151
:101AD000729FBB27F00DB11D639FAA27F00DB11DAA
:101AE000AA1F649F6627B00DA11D661F829F222733
:101AF000B00DA11D621F739FB00DA11D621F839FBA
:101B0000A00D611D221F749F3327A00D611D231F8F
:101B1000849F600D211D822F762F6A2F11249F57DD
:101B200050408AF0E1F088234AF0EE0FFF1FBB1F00
:101B3000661F771F881F91505040A9F79E3F51059F
:101B400070F05CCFA6CF5F3FECF3983EDCF3869558
:101B500077956795B795F795E7959F5FC1F7FE2B4A
:101B6000880F911D9695879597F90895DB018F93BE
:101B70009F930E94020EBF91AF91A29F800D911D75
:101B8000A39F900DB29F900D1124089597FB072EEF
:101B900016F4009407D077FD09D00E94150E07FCBB
:101BA00005D03EF4909581959F4F0895709561956D
:101BB0007F4F0895A1E21A2EAA1BBB1BFD010DC089
:101BC000AA1FBB1FEE1FFF1FA217B307E407F507ED
:101BD00020F0A21BB30BE40BF50B661F771F881FC9
:101BE000991F1A9469F760957095809590959B015F
:101BF000AC01BD01CF010895EE0FFF1F0590F491D8
:101C0000E02D09940E94290EA59F900DB49F900D80
:101C1000A49F800D911D11240895B7FF0C94020E0E
:101C20000E94020E821B930B0895AA1BBB1B51E15D
:101C300007C0AA1FBB1FA617B70710F0A61BB70B3C
:101C4000881F991F5A95A9F780959095BC01CD01E1
:101C50000895A29FB001B39FC001A39F700D811D85
:101C60001124911DB29F700D811D1124911D0895A5
:101C7000FC0188279927E89421912032E9F3293043
:101C800010F02E30C8F32B3241F02D3239F4689425
:101C900004C00E94560E820F911D219120532A30BC
:101CA000C0F31EF4909581959F4F08957AE0979F19
:101CB000902D879F802D910D11240895F894FFCFCA
:101CC00004000400030002000B000A0009000800E1
:101CD0000700060005004750524D43004750474754
:101CE00041004E004E4E4500454E450045534500CF
:101CF0005353450053005353570057535700574E03
:101D000057004E4E570000000000FC09720B7E0980
:061D100097098909DA09B8
:00000001FF
